:100000000C9455060C949C060C949C060C949C062F
:100010000C949C060C949C060C949C060C949C06D8
:100020000C949C060C949C060C9472150C9444162B
:100030000C9445240C949C060C949C060C949C06F1
:100040000C949C060C949C060C949C060C949C06A8
:100050000C949C060C94E5240C949C060C949C0631
:100060000C949C060C94E9080C949C060C949C0639
:100070000C949C060C949C060C949C060C949C0678
:100080000C949C060C949C060C949C060C949C0668
:100090000C949C060C949C060C949C060C949C0658
:1000A0000C949C060C949C060C949C06150E190E40
:1000B0001D0E210E250E290E2D0E310E350E390E78
:1000C0003D0E410E450E490E4D0E510E550E590E68
:1000D0005D0E610E650E690E6D0E710E750E790E58
:1000E0007D0E810E850E890E8D0E910E950E990E48
:1000F0009D0EA10EE10E130EA50EA70EA90EAB0EBE
:10010000AF0EB30EB70EBB0EC00EC50EC90ECD0E90
:10011000D10ED50ED90EDF0EDF0EDF0EDF0EDF0E95
:10012000DF0EDF0EDF0EDF0EDF0EDF0EDF0EDF0E67
:10013000DF0EDF0EDF0EDF0EDF0EDF0EDD0EB1167F
:10014000D316C117D316C11718173B17C11790172D
:10015000A317BA1ABA1AE81AE81A451B831B9C1D82
:100160009C1D9C1B9C1D9D1C9D1C701D9C1D9C1DF5
:10017000871D1F141A16041D1B06202115080709C8
:10018000190522231C170A0B11801E352B39797A89
:100190007B2C2425180C0E0D1080742A31287C7DB0
:1001A0007E7F26271213330F36802D2E302F3438C2
:1001B000378025630025730D0A00522C310D0A008B
:1001C00053592C464646340D0A0053482C303033E0
:1001D000430D0A00537E2C360D0A0053572C38303D
:1001E00030300D0A00534D2C340D0A0053532C4B64
:1001F0006579626F6172642F4D6F7573650D0A00CA
:10020000532D2C546D6B42540D0A0053462C310D66
:100210000A002D2D2D0D0A0045786974696E67203E
:10022000636F6E666967206D6F6465202E2E2E0ADF
:10023000002B0D0A00760D0A0024242400456E745C
:100240006572696E6720636F6E666967206D6F64A3
:1002500065202E2E2E0A00522C310D0A0053522CEE
:100260005A0D0A00555342206D6F64650A004175AE
:10027000746F206D6F64650A00253032750A0025A1
:100280003032753A00253032753A004241543A20F6
:1002900025756D560900757074696D653A202530B5
:1002A000327520253032753A253032753A25303294
:1002B000750A00564255533A2025580A0052656D7A
:1002C0006F746557616B657570456E61626C6564CE
:1002D0003A2025580A000A003F004C4F5700444975
:1002E000534348470043484152470046554C4C0051
:1002F000626174746572793A2000555342205374D8
:100300006174653A2025730A00636F6E6669675FE2
:100310006D6F64653A2025580A00726E34325F6151
:1003200075746F636F6E6E656374696E6728293AC2
:100330002025580A00726E34323A2025730A00666E
:100340006F7263655F7573623A2025580A00707298
:100350006F746F636F6C3A2025730A000A2D2D2D80
:100360002D2D20524E2D343220696E666F202D2D9A
:100370002D2D2D0A00753A20202020202020746F7A
:1003800067676C6520466F72636520555342206D28
:100390006F64650A00703A202020202020207061C0
:1003A0006972696E670A00536C636B3A20202020E3
:1003B000524E2D343220696E697469616C697A65B8
:1003C0000A0044656C3A2020202020656E74657216
:1003D0002F6578697420524E2D343220636F6E661B
:1003E0006967206D6F64650A00623A202020202032
:1003F00020206261747465727920766F6C74616715
:10040000650A00693A20202020202020524E2D34F9
:100410003220696E666F0A000A0A2D2D2D2D2D20BF
:10042000426C7565746F6F746820524E2D343220A3
:1004300048656C70202D2D2D2D2D0A00253032752C
:100440003A253032753A253032750925756D560AD0
:10045000004C4544207374617475733A2025303222
:10046000580A002025303258002563005B735D0078
:100470004B6579626F6172642073746172740A00F3
:10048000524E2D343220696E69740A000A55534267
:1004900020696E69740A005B445D005B435D001275
:1004A00003480048004B00420020006D006F0064CC
:1004B0000000000E0374002E006D002E006B002E55
:1004C0000000000403090409027400040100A032C2
:1004D00009040000010301010009211101000122AA
:1004E00040000705810308000A0904010001030117
:1004F0000200092111010001224D000705820308B5
:10050000000A090402000103000000092111010092
:10051000012236000705830308000A0904030002CC
:1005200003000000092111010001222200070584B7
:10053000032000010705040320000112011001003F
:10054000000008EDFE42420401010200010631FFF5
:100550000974A1010975150026FF00952075088111
:10056000020976150026FF00952075089102C00546
:10057000010980A101850216810026B7001A8100B9
:100580002AB700751095018100C0050C0901A10171
:100590008503160100269C021A01002A9C02751090
:1005A00095018100C005010902A1010901A1000511
:1005B0000919012905150025019505750181029587
:1005C00001750381010501093009311581257F95E8
:1005D000027508810609381581257F950175088106
:1005E00006050C0A38021581257F950175088106DC
:1005F000C0C005010906A101050719E029E715009A
:10060000250195087501810295017508810105088C
:10061000190129059505750191029501750391014F
:100620000507190029FF150026FF009506750881AA
:1006300000C0636F6E73756D65723A202530345853
:100640000A0073797374656D3A20253034580A00B6
:100650000A002530325820006B6579626F61726440
:100660003A20004C45443A20253032580A002530C3
:1006700032583A202530386225730A00722F6320E1
:1006800030313233343536370A004F6E6573686F58
:10069000743A2074696D656F75740A00290A002523
:1006A00075002F002575005D2800256400200025B9
:1006B0006400200025640020002564007C002530B3
:1006C0003258006D6F7573656B6579205B62746E6F
:1006D0007C782079207620685D287265702F6163B0
:1006E0006C293A205B006D6B5F776865656C5F74A1
:1006F000696D655F746F5F6D6178203D2025640AC8
:10070000006D6B5F776865656C5F6D61785F7370B6
:10071000656564203D2025640A006D6B5F74696D1A
:10072000655F746F5F6D6178203D2025640A006D00
:100730006B5F6D61785F7370656564203D20256433
:100740000A006D6B5F696E74657276616C203D2086
:1007500025640A006D6B5F64656C6179203D20251E
:10076000640A006D6B5F776865656C5F74696D65C1
:100770005F746F5F6D6178203D2025640A006D6BAA
:100780005F776865656C5F6D61785F7370656564E0
:10079000203D2025640A006D6B5F74696D655F7490
:1007A0006F5F6D6178203D2025640A006D6B5F6D81
:1007B00061785F7370656564203D2025640A006D73
:1007C0006B5F696E74657276616C203D2025640AEA
:1007D000006D6B5F64656C6179203D2025640A00C3
:1007E0000A00257500363A20776865656C5F746984
:1007F0006D655F746F5F6D61783A20000A00257542
:1008000000353A20776865656C5F6D61785F73705D
:100810006565643A20000A00257500343A20746941
:100820006D655F746F5F6D61783A20000A00257511
:1008300000333A206D61785F73706565643A20001B
:100840000A00257500323A20696E74657276616C13
:10085000286D73293A20000A00257500313A20647A
:10086000656C6179282A31306D73293A20000A09B4
:100870002D2056616C756573202D0A004D3E004D8C
:1008800025643E20003F00736574206465666175D1
:100890006C740A00433E20007768657265206465C9
:1008A0006C74613A20637572736F723D25642C20FD
:1008B000776865656C3D25640A53656520687474C6
:1008C000703A2F2F656E2E77696B69706564696168
:1008D0002E6F72672F77696B692F4D6F7573655F28
:1008E0006B6579730A000A092D204D6F7573656B6E
:1008F0006579202D0A4553432F713A097175697442
:100900000A313A0964656C6179282A31306D73299E
:100910000A323A09696E74657276616C286D7329C2
:100920000A333A096D61785F73706565640A343A19
:100930000974696D655F746F5F6D61780A353A0996
:10094000776865656C5F6D61785F73706565640A73
:10095000363A09776865656C5F74696D655F746FB9
:100960005F6D61780A0A703A097072696E74207658
:10097000616C7565730A643A097365742064656611
:1009800061756C74730A75703A092B310A646F775C
:100990006E3A092D310A706775703A092B31300AA9
:1009A0007067646F776E3A092D31300A0A7370658B
:1009B0006564203D2064656C7461202A206D617837
:1009C0005F7370656564202A2028726570656174A4
:1009D000202F2074696D655F746F5F6D6178290ADF
:1009E000003F004D3E2000433E20004C25640A009D
:1009F0000A092D20436F6E736F6C65202D0A4553D5
:100A0000432F713A09717569740A6D3A096D6F75F2
:100A100073656B65790A000A092D204D616769636A
:100A2000202D0A643A0964656275670A783A096498
:100A300065627567206D61747269780A6B3A096442
:100A400065627567206B6579626F6172640A6D3AE1
:100A5000096465627567206D6F7573650A763A097A
:100A600076657273696F6E0A733A0973746174758F
:100A7000730A633A09636F6E736F6C65206D6F6400
:100A8000650A302D343A096C61796572302D34284D
:100A90004631302D4634290A506175733A09626F28
:100AA0006F746C6F616465720A003F0074696D65F4
:100AB000725F72656164333228293A202530346CC4
:100AC000580A006B6579626F6172645F69646C6576
:100AD0003A2025580A006B6579626F6172645F7015
:100AE000726F746F636F6C3A2025580A00686F73D9
:100AF000745F6B6579626F6172645F6C65647328A3
:100B0000293A2025580A000A092D2053746174756A
:100B100073202D0A004743433A20342E392E3220C9
:100B20004156522D4C4942433A20312E382E3073D3
:100B3000766E204156525F415243483A20617672A8
:100B4000350A004F5054494F4E533A204C554641B8
:100B5000204D4F5553454B45592045585452414B14
:100B6000455920434F4E534F4C4520434F4D4D4127
:100B70004E44204B45594D41505F53454354494FD6
:100B80004E20343039360A004255494C443A20351B
:100B90003732633236352D646972747920283134E6
:100BA0003A33303A3232204A616E203235203230C8
:100BB0003137290A005649443A20307846454544A1
:100BC00028742E6D2E6B2E29205049443A203078FF
:100BD000343234322848484B42206D6F6429205605
:100BE00045523A203078303130340A00444553437E
:100BF0003A20742E6D2E6B2E206B6579626F6172B8
:100C000064206669726D7761726520666F72204834
:100C1000484B42206D6F640A000A092D2056657208
:100C200073696F6E202D0A000A6D6F7573653A2027
:100C30006F66660A000A6D6F7573653A206F6E0AFB
:100C4000000A6B6579626F6172643A206F66660AAA
:100C5000000A6B6579626F6172643A206F6E0A00F8
:100C60000A6D61747269783A206F66660A000A6DCF
:100C700061747269783A206F6E0A000A6465627561
:100C8000673A206F6E0A000A64656275673A206FE2
:100C900066660A000A0A626F6F746C6F616465723F
:100CA0002E2E2E2000433E20000011241FBECFEF29
:100CB000DAE0DEBFCDBF04B603FE27C080915F033C
:100CC00090916003A0916103B09162038730904BD3
:100CD000A740B04BD1F410925F03109260031092C2
:100CE00061031092620314BE84B7877F84BF0FB67E
:100CF000F894A895809160008861809360001092BC
:100D000060000FBEE0E0F8E3099511E0A0E0B1E07B
:100D1000ECEDFAE502C005900D92AA39B107D9F7BA
:100D200023E0AAE9B1E001C01D92AF35B207E1F7B7
:100D30000E941C100C946C2D0C9400000FB6809532
:100D40009AE0F8947BE27A95F1F708F0589A08F463
:100D5000589886959A95B1F70FBE08950FB680E81A
:100D6000F894499BFECF4999FECF96E19A95F1F709
:100D70009CE29A95F1F7869549998068C8F70FBE6D
:100D800008950FB680E8F89496E19A95F1F79CE201
:100D90009A95F1F7869549998068C8F796E19A95F2
:100DA000F1F7499BFECF0FBE0895FF93EF93E091BB
:100DB0009A01F0919B01309709F00995EF91FF910D
:100DC0000895FC018591803011F0EFDFFBCF08958D
:100DD000FF27E0E230E247FF0CC0419597FF09C0D2
:100DE000EDE26095709580959095611D711D811D56
:100DF000911D27FF02C0219530E350E2AA27660F1C
:100E0000771F881F991FAA1FA41710F0A41B6395B2
:100E10005A95A9F7AA3008F0A95FA05DAF93F395A2
:100E2000611571058105910541F7ED3211F4EF93DC
:100E3000F395F21718F43F93F395FBCF8F91B5DF3D
:100E4000FA95E1F70895E991F9918591803021F0C3
:100E5000853219F0AADFF9CF089520E0E894559182
:100E60005532C1F3503311F4689455915A3348F414
:100E7000505390F3220F022E220F220F200D250F28
:100E8000F4CF0EF4219589919991533619F3533784
:100E900029F1533559F1BC0188279927E8945C362C
:100EA00021F48991999168945591543639F446EF1B
:100EB0007EF077FF0DC08FEF9FEF0AC055374AE0F5
:100EC00039F0583540E121F0523642E009F00895FA
:100ED000FF93EF937DDFEF91FF91B7CFFF93EF93F8
:100EE000FC0181918030B9F360DFFBCFFF93EF937A
:100EF00068DFF1CFDF93CF93CDB7DEB72596A3DFC1
:100F0000CF91DF91089514B88FEF85B9549A5C980A
:100F100008958FEF84B980E485B9549A5C9A8FE183
:100F20009EE40197F1F700C0000008958FEF84B9A7
:100F300080E485B957985F9A87B18F7387B988B174
:100F4000806C88B92E9A2F980E948307E4EAF1E01A
:100F500088E08E0F11928E13FDCFECE9F1E088E06E
:100F60008E0F11928E13FDCF84EA91E09093AF0122
:100F70008093AE018CE991E09093AD018093AC0138
:100F800008950F931F93CF93DF938091AC019091BD
:100F9000AD012091AE013091AF013093AD012093AE
:100FA000AC019093AF018093AE015C9B0E948907D6
:100FB000C0E0D0E001E010E080E090E025B1207CCE
:100FC0002C2BAC0133E0440F551F3A95E1F7242B4D
:100FD00025B9EAE1EA95F1F700C0E091AC01F091A2
:100FE000AD01EC0FFD1F208130E0082E02C03595C9
:100FF00027950A94E2F720FD2F9AF5E3FA95F1F789
:101000000000E6B52E982AE12A95F1F700C040913C
:10101000AE015091AF01DA01AC0FBD1F4F9B0AC06A
:101020009801082E01C0220F0A94EAF720953C91FE
:10103000232308C06C919801082E01C0220F0A9446
:10104000EAF7262B2C9326B56E2F70E02E1718F09A
:1010500026B530E004C026B530E021503F4F261BB6
:10106000370B2630310558F0E091AC01F091AD011D
:10107000EC0FFD1F2081FA01EC0FFD1F20833AE1E8
:101080003A95F1F700C02F982E9AEBE2F1E03197F4
:10109000F1F700C0000001968830910509F08ECF6D
:1010A000A091AE01B091AF01AC0FBD1FE091AC01BA
:1010B000F091AD01EC0FFD1F9C918081981751F0CC
:1010C0000E9483246093B0017093B1018093B201B8
:1010D0009093B3012196C830D10509F06DCF5C9B88
:1010E0001BC080915603853021F0809156038111F9
:1010F00013C06091B0017091B1018091B2019091E3
:10110000B3010E94B924613177428105910520F035
:101110000E9483070E94042481E0DF91CF911F91F8
:101120000F9108952091AE013091AF01F901E80FC0
:10113000F11D808108950C9489070C948307569AB9
:1011400081FF02C05E9A08955E98089588E08093BA
:10115000CC001092CD00E9ECF0E0808180698083C2
:10116000808188608083EAECF0E080818083EBEC12
:10117000F0E080818083559A5D98789408959091ED
:10118000B5012091B4019217D1F030E0F901EA5491
:10119000FE4F80812F5F3F4F33272093B401492FAB
:1011A00050E0921718F4241B350B03C0241B350B99
:1011B0003395233031050CF05D9890E008958FEF62
:1011C0009FEF08959091C80095FFFCCF8093CE00CB
:1011D00008951F920F920FB60F9211242F933F93F1
:1011E0004F935F938F939F93EF93FF938091B501FC
:1011F00090E0AC014F5F5F4F2091B401241741F0A4
:101200003091CE00FC01EA54FE4F30834093B5018B
:101210003091B501822F90E0432F50E0841B950B55
:10122000321708F0939503970CF45D9AFF91EF91B4
:101230009F918F915F914F913F912F910F900FBE92
:101240000F901F9018958091D00208950895809175
:10125000D00208950895089508950895CF93DF93D7
:101260008D3C9105B9F1B8F4853B9105A9F148F49D
:10127000833B9105D1F1843B9105D1F5D0E0C0E2EB
:101280003BC0873B910571F150F18C3C910581F594
:10129000D0E0C8E031C08A3E9105C1F040F4823E02
:1012A0009105B1F0893E910519F5D0E124C0813254
:1012B00022E0920749F0833222E09207D9F08A387F
:1012C0009140B1F4D2E017C0D4E015C0D0E213C011
:1012D000D0E411C0D0E80FC0D0E0C1E00DC0D0E034
:1012E000C2E00AC0D0E0C4E007C0D0E0C0E104C062
:1012F000D0E001C0D1E0C0E08DEF0E94E20883E0C1
:101300000E94E20883E00E94E2088D2F0E94E2081A
:101310008C2FDF91CF910C94E208CF93DF93EC01F7
:101320008DEF0E94E20885E00E94E20882E00E94C0
:10133000E20888810E94E20889810E94E2088A818D
:101340000E94E2088B81DF91CF910C94E208CF9349
:10135000DF93EC018DEF0E94E20889E00E94E20831
:1013600081E00E94E20888810E94E20880E00E94F9
:10137000E2088A810E94E2088B810E94E2088C8147
:101380000E94E2088D810E94E2088E810E94E2089C
:101390008F81DF91CF910C94E2080C94BF08EF92FB
:1013A000FF920F931F93CF938C010E9477247C01AF
:1013B000C0E0C7010E948F248017910798F40E9413
:1013C000BF089C012F3F8FEF380751F02D3041F0BF
:1013D0002A3041F0EC2FF0E0E854FD4F2083CF5F3E
:1013E000C73138F3EC2FF0E0E854FD4F108288EB62
:1013F00092E0CF911F910F91FF90EF9008950C9480
:10140000E20881B3881F8827881F0895879A8F9ADA
:10141000089585B7806885BF85B7806885BF0E94BD
:10142000060A86988E9A81988998559A5D980C94A8
:10143000A608879A8F9808958FB186958170089530
:101440008FB186FB882780F908958093D002089594
:10145000CF93DF93FC018491EF012196882321F043
:101460000E94E208FE01F7CFDF91CF910895CF935C
:10147000DF93C2EBD1E00E94BF088F3F2FEF9207AE
:1014800059F09F938F93DF93CF930E947A070F9029
:101490000F900F900F90EFCFDF91CF9108950E94A2
:1014A000280A2FEF89E698E1215080409040E1F72B
:1014B00000C0000084E690E00E94CF098093B6024D
:1014C0009093B7029F938F9385EB91E09F938F93B7
:1014D0000E947A070E94370A0F900F900F900F908A
:1014E0008091B6029091B70208950E94DE17909302
:1014F0001501809314010E94BE1D80E091E00E94BE
:10150000D9170E94190A0E94200A8111FCCF8DE38D
:1015100092E00E94E1062FEF85EB95E32150804099
:101520009040E1F700C0000089E392E00E944F0A7A
:10153000EFEFFBE42DE1E150F0402040E1F700C087
:1015400000000E94370A85E392E00E944F0AFC01E6
:101550008081863721F081E392E00C944F0A089550
:1015600088E192E00E94E10682E192E00E944F0A47
:101570000E94060A0E94BE1D8091140190911501DF
:101580000C94D9170C94580F8F929F92AF92BF92E0
:10159000CF92DF92EF92FF920F931F93CF93DF933F
:1015A00092E0B92E03E614E029E6E22E24E0F22EC2
:1015B000AA24A39433E0932E41E5C42E44E0D42E14
:1015C0000E94CD09EC01019609F441C08091D3023B
:1015D0008130F9F028F0823009F1833021F134C0F4
:1015E000CE3FD10519F4A092D302EACFC038D1057D
:1015F00028F4DF93CF93FF92EF9204C0DF93CF9351
:101600001F930F930E947A070F900F900F900F90E7
:10161000D7CF2297C9F4B092D302D2CF2197A1F4A9
:101620009092D302CDCF8091410380FF0AC0DF9317
:10163000CF93DF92CF920E947A070F900F900F9076
:101640000F908C2F0E94250A1092D302B9CF80915F
:10165000D502811121C08091D40281111DC00E9448
:101660001C0A81110AC00E94DE178A50914029F09D
:101670000E94BE1D8AE091E00DC00E941C0A8823D2
:1016800059F00E94DE178651914031F00E94BE1D34
:1016900086E191E00E94D9178091D1029091D20207
:1016A0000E948F24893E23E0920708F461C028EE4F
:1016B00033E0B9010E941C2D629FC001639F900D11
:1016C000729F900D11242091D1023091D202820F8D
:1016D000931F9093D2028093D1020E94F60F833021
:1016E00011F481E001C080E00E94470F0E94832432
:1016F00028EE33E040E050E00E94442D49015A01B9
:101700008CE3C82ED12CE12CF12CCA01B901A70120
:1017100096010E94442D672B682B692B49F50E9486
:10172000BF0F2091410320FF23C09F938F931F92EF
:101730001F92C501B40120E13EE040E050E00E946C
:10174000442DC22FA70196010E94442D3F932F9351
:101750001F92CF938CE394E09F938F930E947A071C
:101760008DB79EB70A960FB6F8949EBF0FBE8DBF79
:101770000E941C0A811107C00E94200A882319F0C8
:101780006E9A769802C06E9A769ADF91CF911F91E9
:101790000F91FF90EF90DF90CF90BF90AF909F9010
:1017A0008F9008958F929F92AF92BF92CF92DF92C7
:1017B000EF92FF921F93CF93DF9300D000D0CDB76D
:1017C000DEB7833109F48CC008F05BC08B3009F4BC
:1017D00066C08C3009F48FC0853009F0FBC10E94CF
:1017E000832428EE33E040E050E00E94442D49017C
:1017F0005A010E94BF0F9F938F938BE892E09F93B3
:101800008F930E947A07C501B40120E13EE040E0D9
:1018100050E00E94442D5F934F933F932F9325E810
:1018200032E03F932F9369837A838B839C830E945A
:101830007A078CE3C82ED12CE12CF12C69817A81B6
:101840008B819C81A70196010E94442D5F934F9349
:101850003F932F938FE792E09F938F930E947A0795
:10186000C501B401A70196010E94442D9F938F9357
:101870007F936F9389E792E09F938F930E947A07FB
:1018800040C1883361F020F4883109F440C1A2C11D
:10189000873409F46DC18C3409F456C19BC188E1C9
:1018A00094E00E94E10683E094E00E94E10689EE64
:1018B00093E00E94E10682EC93E00E94E10687EA51
:1018C00093E00E94E10685E993E00E94E106109111
:1018D000D50211117DC185E793E00E94E1067EC12A
:1018E0000E94750A8DE592E00E944F0A87E592E01A
:1018F0000E944F0A6BC18CE593E00E94E1060E94B2
:10190000DE178A50914019F08FE291E002C089E21F
:1019100091E09F938F938EE493E09F938F930E9427
:101920007A078091D4021F928F938FE393E09F9365
:101930008F930E947A070E941C0A0FB6F894DEBFAC
:101940000FBECDBF811107C00E94200A811106C0C1
:1019500088E391E005C084E391E002C08BE391E06D
:101960009F938F9385E393E09F938F930E947A07D1
:101970000E94010A1F928F938AE193E09F938F93B5
:101980000E947A078091D5021F928F9389E093E09D
:101990009F938F930E947A07809156030FB6F89415
:1019A000DEBF0FBECDBF8823B9F0809156038130D2
:1019B000B1F0809156038230A9F0809156038330B4
:1019C000A1F080915603843099F0809156038530C0
:1019D00091F080E791E011C088E491E00EC080E4CE
:1019E00091E00BC083E591E008C08BE591E005C074
:1019F00085E691E002C082E791E09F938F938AEFA2
:101A000092E09F938F930E947A0780EF92E09F93DA
:101A10008F930E947A070E94F60F0F900F900F90FD
:101A20000F900F900F90813059F038F0823059F0BC
:101A3000833061F48AED92E00BC08BEE92E008C037
:101A400085EE92E005C08EED92E002C088ED92E056
:101A50009F938F930E947A070F900F9086ED92E0EC
:101A60009F938F930E947A07809154031F928F93C4
:101A70008DEB92E09F938F930E947A078091D9001B
:101A800081701F928F9383EB92E09F938F930E94BC
:101A90007A070E94832428EE33E040E050E00E9461
:101AA000442D69017A019CE3892E912CA12CB12C43
:101AB000CA01B901A50194010E94442D7F936F933F
:101AC000C701B60120E13EE040E050E00E94442D15
:101AD000122FA50194010E94442D3F932F931F9232
:101AE0001F93C701B60120E831E541E050E00E94B4
:101AF000442D3F932F9386E992E09F938F930E940A
:101B00007A070FB6F894DEBF0FBECDBF61C08091DB
:101B1000D502811162C01091D402112339F08EE6F2
:101B200092E00E94E1061092D40258C084E692E04E
:101B30000E94E10681E08093D4020E94BE1D86E1EE
:101B400091E00E94D91744C00E94010A182F8823EF
:101B500041F00E94750A81E0809351038093D50281
:101B60003DC00E94B00A109251031092D50230C0BD
:101B70008091D502811102C00E94750A8BE092E02B
:101B80000E944F0A80E092E00E944F0A8CEE91E0A2
:101B90000E944F0A85EE91E00E944F0A8BED91E082
:101BA0000E944F0A84ED91E00E944F0A8AEC91E076
:101BB0000E944F0A80EC91E00E944F0A8AEB91E06C
:101BC0000E944F0A8091D502811102C00E94B00A82
:101BD00011E004C01091D50201C010E0812F0F90D8
:101BE0000F900F900F90DF91CF911F91FF90EF908A
:101BF000DF90CF90BF90AF909F908F900895CF933C
:101C0000C82F0E943923827291E009F490E04C2F92
:101C100050E0FA013497E934F10508F0D0C0EA5AEF
:101C2000FF4F0C94662D8BE12DC19111CCC081E644
:101C300029C19111CAC082E625C19111C8C083E6AD
:101C400021C19111C6C084E61DC19111C4C085E6B1
:101C500019C19111C2C086E615C19111C0C087E6B5
:101C600011C19111BEC088E60DC19111BCC089E6B9
:101C700009C19111BAC08AE605C19111B8C08BE6BD
:101C800001C19111B6C08CE6FDC09111B4C08DE6C2
:101C9000F9C09111B2C08EE6F5C09111B0C08FE6C7
:101CA000F1C09111AEC080E7EDC09111ACC081E7E9
:101CB000E9C09111AAC082E7E5C09111A8C083E7ED
:101CC000E1C09111A6C084E7DDC09111A4C085E7F1
:101CD000D9C09111A2C086E7D5C09111A0C087E7F5
:101CE000D1C091119EC088E7CDC091119CC089E7F9
:101CF000C9C091119AC08AE7C5C0911198C081E30B
:101D0000C1C0911196C082E3BDC0911194C083E31C
:101D1000B9C0911192C084E3B5C0911190C085E320
:101D2000B1C091118EC086E3ADC091118CC087E324
:101D3000A9C091118AC088E3A5C0911188C089E328
:101D4000A1C0911186C080E39DC088E09BC089E05E
:101D500099C080E297C091117EC08DE293C091112D
:101D60007CC08DE38FC091117AC08BE58BC091113F
:101D700078C08DE587C0992309F475C08CE782C0CF
:101D8000992309F472C08CE77DC0911170C08BE378
:101D900079C091116EC087E275C091116CC080E668
:101DA00071C091116AC08CE26DC0911168C08EE261
:101DB00069C0911166C08FE265C080E063C080E2B7
:101DC00061C08AE05FC081E45DC082E45BC083E4FF
:101DD00059C084E457C085E455C086E453C087E405
:101DE00051C088E44FC089E44DC08AE44BC08BE405
:101DF00049C08CE447C08DE445C08EE443C08FE405
:101E000041C080E53FC081E53DC082E53BC083E540
:101E100039C084E537C085E535C086E533C087E540
:101E200031C088E52FC089E52DC08AE52BC081E24D
:101E300029C080E427C083E225C084E223C085E274
:101E400021C08EE51FC086E21DC08AE21BC088E269
:101E500019C089E217C08FE515C08BE213C08BE76C
:101E600011C08DE70FC08CE50DC08CE50BC08AE377
:101E700009C082E207C08EE705C08CE303C08EE391
:101E800001C08FE30E94FF0981E0CF910895833064
:101E900019F4859A7D9A0895813011F4859A06C0C7
:101EA000823019F4859A8D9A089585988D980895B1
:101EB00081E00E94470F2FEF81EE94E02150804097
:101EC0009040E1F700C0000082E00E94470F2FEF32
:101ED00081EE94E0215080409040E1F700C0000086
:101EE00081E00E94470F2FEF81EE94E02150804067
:101EF0009040E1F700C0000082E00E94470F2FEF02
:101F000081EE94E0215080409040E1F700C0000055
:101F100080E00E94470F80EC80937C0087E08093F4
:101F20007A0081E980937E0081E080937F008BE3DB
:101F300080937D00849A8C9808958091D90080FFC9
:101F40001CC090B331B385988D9AEFE9FFE03197CB
:101F5000F1F700C000008FB185FB882780F920B31E
:101F600090722F7D292B20BB91B3232F20729F7D50
:101F7000922B91BB91E08927089580E00895CF933B
:101F8000DF9300D0CDB7DEB7849A8C9A80917A0027
:101F9000806880937A008FE99FE00197F1F700C095
:101FA000000080917A00806480937A0080917A00AA
:101FB00086FDFCCF80917800909179009A83898387
:101FC00080917A008F7780937A00849A8C98298107
:101FD0003A8145E0429FC001439F900D11248055F6
:101FE00091090F900F90DF91CF9108958091D900C2
:101FF00080FD0C949D0F0E94BF0F8C3A2DE092073C
:1020000020F481E08093D60205C085379E4010F011
:102010001092D6028091D602811102C082E008950A
:1020200083E00895CF93C82F0E949E068C2F0E94B4
:102030009F1080E0CF91089584B7877F84BF0FB64B
:10204000F894A89580916000886180936000109258
:1020500060000FBE90E080E80FB6F89480936100B6
:10206000909361000FBE0E94F7140E945415809156
:10207000E20084608093E20082E190E10E94D52337
:10208000509A589A5198599A78948FEF9091560394
:102090008150943041F0EFE7FEE33197F1F700C053
:1020A00000008111F3CF8CE894E00E94E1060E94C9
:1020B000090A0E94C20A80E894E00E94E1060E9498
:1020C0009F180E941C0A811103C08AE091E002C09F
:1020D00086E191E00E94D91780E794E00E94E10632
:1020E0000E941C0A882319F1809156038530F9F467
:1020F0008CE694E00E94E1060E949D080E94042460
:102100000E9404240E9404240E9404240E940424A7
:102110000E9404240E94042480915403882301F324
:102120000E942D248823E1F20E944C13D9CF0E94F3
:10213000A3180E94C40AD4CF8091E30208959FB7E8
:10214000F8941092DA029FBF90915603943009F0F0
:1021500057C09091E9009F703091EC00232F2170BF
:1021600030FD20E8922B24E02093E9002091EB0041
:1021700020FF43C02091EE0027FF3FC02091D702EF
:10218000222321F02091E80025FF37C01092D702CA
:1021900026E03091E80035FD15C03091560334300B
:1021A00061F53091EB0035FD28C0215021F481E02C
:1021B0008093D70222C0EFE9FFE03197F1F700C02A
:1021C0000000E7CF8093F1008091E80085FD0AC010
:1021D0008091E80080FFFCCF8091E8008E778093AB
:1021E000E80006C08FB7F89421E02093DA028FBF91
:1021F0009F709093E90080E008959F709093E900AC
:102200008FEF0895CF93DF9300D01F92CDB7DEB745
:102210009C0180915603843019F593E099833B83A8
:102220002A839093E9008FEF9091E800815095FD0B
:1022300006C095ED9A95F1F700008111F5CF8091D8
:10224000E80085FF0DC040E050E063E070E0CE01A3
:1022500001960E9462138091E8008E778093E800D7
:102260000F900F900F90DF91CF910895CF93DF9350
:1022700000D01F92CDB7DEB720915603243021F550
:1022800022E029839B838A8383E08093E9008FEF98
:102290009091E800815095FD06C095ED9A95F1F773
:1022A00000008111F5CF8091E80085FF0DC040E06E
:1022B00050E063E070E0CE0101960E9462138091CD
:1022C000E8008E778093E8000F900F900F90DF91D9
:1022D000CF910895209156032430F1F422E0209309
:1022E000E9002FEF3091E800215035FD06C035EDB3
:1022F0003A95F1F700002111F5CF2091E80025FF74
:102300000BC040E050E065E070E00E9462138091F5
:10231000E8008E778093E8000895CF93DF932091B3
:102320005603243039F521E02093E9002FEF309156
:10233000E800215035FD06C035ED3A95F1F7000073
:102340002111F5CF2091E80025FF14C0EC0140E0F9
:1023500050E068E070E00E9462138091E8008E77A0
:102360008093E80088E0FE01ABEDB2E001900D92B1
:102370008A95E1F7DF91CF9108958BE994E00E946F
:10238000E10680915503811109C00E94F7140E9453
:1023900054158091E20084608093E200089587E9FB
:1023A00094E00E94E106109255030895089520914B
:1023B000D8022F5F822F62E30E94102D992319F01B
:1023C0002093D80208951092D8028091DA028823CF
:1023D00071F180915603843041F58091E9008F704E
:1023E0002091EC00922F917020FD90E8892B94E0D1
:1023F0009093E9009091EB0090FF14C09091EE0053
:1024000097FF10C09091E80095FF03C01092F10073
:10241000F9CF9091E80090FF05C09091E8009E7779
:102420009093E8008F708093E9001092DA0208958B
:1024300042E061EC81E00E94711442E061EC82E0D4
:102440000E94711442E061EC83E00E94711442E248
:1024500061EC84E00C94711480915803833009F48A
:1024600053C030F4813071F0823009F48CC008958B
:102470008A3009F478C08B3009F45EC0893009F0E5
:102480009AC020C080915703813A09F094C080918E
:10249000E800877F8093E80080915B0390915C0364
:1024A000892B21F468E08BED92E003C060E080E0CE
:1024B00090E070E00E94AD138091E8008B778093EC
:1024C000E800089580915703813209F074C080912B
:1024D0005B0390915C03892B09F06DC08091E8004B
:1024E000877F8093E8008091E80082FD05C080919D
:1024F00056038111F8CF5FC08091F1008093E30211
:102500008091E8008B7753C080915703813A09F09E
:1025100052C080915B0390915C03892B09F04BC002
:102520008091E800877F8093E8008091E80080FF39
:10253000FCCF8091200136C0809157038132D9F5BC
:1025400080915B0390915C03892BA9F58091E80051
:10255000877F8093E8000E94A6148091590380939E
:1025600020010C94BE1D80915703813221F580918A
:10257000E800877F8093E8000E94A61480915A03A8
:102580008093E402089580915703813AA1F48091E9
:10259000E800877F8093E8008091E80080FFFCCF0F
:1025A0008091E4028093F1008091E8008E7780931F
:1025B000E8000C94A61408958091E3028093D90258
:1025C0001092E30280E00E949F080E9462190C941E
:1025D000BE1D0C94DC120E9441248091D90280938C
:1025E000E30208950C94EB12292F33272330310591
:1025F000C9F064F42130310581F02230310509F051
:1026000043C084E790E027EC34E042C0213231053A
:10261000F1F02232310541F137C082E190E02BE345
:1026200035E036C099278130910541F0823091051F
:1026300041F0892B49F5E3ECF4E005C0E3EBF4E06D
:1026400002C0EFE9F4E0849190E09F0121C0643082
:10265000D8F4E62FF0E0EE0FFF1FE857FE4F208181
:10266000318189E090E014C0643070F470E0FB01C7
:10267000EE0FFF1FE058FE4F20813181FB01E4582F
:10268000FE4F808190E004C080E090E020E030E0E8
:10269000FA0131832083089580E189BD82E189BDFB
:1026A00009B400FEFDCF8091D8008F7D8093D800C3
:1026B0008091E00082608093E0008091E00081FDE5
:1026C000FCCF0895CF92DF92EF92FF920F931F936A
:1026D000CF93DF93EC018B016A010E94C514811135
:1026E00033C0C114D10439F0F60180819181081BF7
:1026F000190BC80FD91FE12CF12C0115110519F187
:102700008091E80085FD16C08091E8008E77809367
:10271000E800C114D10449F0F60180819181E80EEE
:10272000F91EF182E08285E00FC00E94C514882363
:1027300021F30AC089918093F10001501109FFEF44
:10274000EF1AFF0ADACF80E0DF91CF911F910F914E
:10275000FF90EF90DF90CF90089520915D0330912E
:102760005E032617370748F06115710539F420918B
:10277000E8002E772093E80001C0B90140E0611520
:102780007105A9F120915603222309F443C0253095
:1027900009F442C02091E80023FD40C02091E800E8
:1027A00022FD32C02091E80020FFE9CF4091F300E4
:1027B0002091F20030E0342BFC01CF01611571054E
:1027C00059F02830310540F481918093F100615037
:1027D00071092F5F3F4FF1CF41E02830310509F0FB
:1027E00040E02091E8002E772093E800C8CF411107
:1027F000C9CF0AC080915603882361F0853061F00B
:102800008091E80083FD0AC08091E80082FFF2CF4A
:1028100080E0089582E0089583E0089581E00895BE
:1028200020915D0330915E032617370748F061154C
:10283000710539F42091E8002E772093E80001C05B
:10284000B901FC0120E06115710591F180915603F9
:10285000882309F440C0853009F43FC08091E80026
:1028600083FD3DC08091E80082FD2FC08091E8008B
:1028700080FFE9CF2091F3008091F20090E0922B4D
:102880006115710559F08830910540F42491209329
:10289000F1003196615071090196F2CF21E008975D
:1028A00009F020E08091E8008E778093E800CBCF9C
:1028B0002111CCCF0AC080915603882361F0853066
:1028C00061F08091E80083FD0AC08091E80082FFFA
:1028D000F2CF80E0089582E0089583E0089581E0DA
:1028E0000895982F973058F59093E900981739F08C
:1028F0007091EC002091ED005091F00003C0242F66
:10290000762F50E021FF19C03091EB003E7F3093CD
:10291000EB003091ED003D7F3093ED003091EB0006
:1029200031603093EB007093EC002093ED005093F6
:10293000F0002091EE0027FF07C09F5FD3CF8F707C
:102940008093E90081E0089580E008958091570325
:1029500087FF11C08091E80082FD05C08091560379
:102960008111F8CF11C08091E8008B770BC0809166
:102970005603882349F08091E80080FFF8CF8091CA
:10298000E8008E778093E80008952091E40030916C
:10299000E50095E64091EC00842F817040FF22C055
:1029A0008091E80080FD1CC080915603882391F03F
:1029B000853091F08091EB0085FD10C04091E400DE
:1029C0005091E5004217530729F39A01915011F7EE
:1029D00084E0089582E0089583E0089581E00895F9
:1029E00080E008954091E80042FFDECF08950E9404
:1029F00065150E946D15E0EEF0E0808181608083B6
:102A0000E8EDF0E080818F77808319BCA7EDB0E01E
:102A10008C918E7F8C9380818F7E80831092550362
:102A200008950F931F93CF93DF930E9465150E9423
:102A30006D15C8EDD0E088818F77888388818068A4
:102A4000888388818F7D888319BC109256031092E9
:102A50005203109254031092530300EE10E0F80159
:102A600080818B7F808388818160888342E060E001
:102A700080E00E947114E1EEF0E080818E7F80831F
:102A8000E2EEF0E0808181608083808188608083D5
:102A9000F80180818E7F8083888180618883DF91C7
:102AA000CF911F910F910895E8EDF0E080818F7E26
:102AB0008083E7EDF0E080818160808384E082BFE5
:102AC00081E0809355030C941115E8EDF0E08081CE
:102AD0008E7F80831092E20008951092DA001092A7
:102AE000E10008951F920F920FB60F9211242F93B9
:102AF0003F934F935F936F937F938F939F93AF9386
:102B0000BF93EF93FF938091E10082FF0BC0809110
:102B1000E20082FF07C08091E1008B7F8093E1009B
:102B20000E94D7118091DA0080FF1FC08091D800E9
:102B300080FF1BC08091DA008E7F8093DA00809145
:102B4000D90080FF0DC080E189BD82E189BD09B453
:102B500000FEFDCF81E0809356030E94BD1105C0A9
:102B600019BC109256030E94CF118091E10080FFA2
:102B700019C08091E20080FF15C08091E2008E7F35
:102B80008093E2008091E20080618093E200809176
:102B9000D80080628093D80019BC85E080935603EA
:102BA0000E94E9128091E10084FF30C08091E20030
:102BB00084FF2CC080E189BD82E189BD09B400FE9B
:102BC000FDCF8091D8008F7D8093D8008091E10067
:102BD0008F7E8093E1008091E2008F7E8093E200FF
:102BE0008091E20081608093E2008091520388230B
:102BF00011F084E007C08091E30087FD02C081E00E
:102C000001C083E0809356030E94F2128091E1009C
:102C100083FF29C08091E20083FF25C08091E100FD
:102C2000877F8093E10082E08093560310925203E5
:102C30008091E1008E7F8093E1008091E2008E7FA1
:102C40008093E2008091E20080618093E20042E0A4
:102C500060E080E00E9471148091F00088608093B1
:102C6000F0000E94D611FF91EF91BF91AF919F911B
:102C70008F917F916F915F914F913F912F910F9025
:102C80000FBE0F901F9018951F920F920FB60F92C4
:102C900011242F933F934F935F936F937F938F9361
:102CA0009F93AF93BF93CF93DF93EF93FF93C09125
:102CB000E900CF708091EC00D82FD17080FDD0E872
:102CC0001092E9008091F000877F8093F000789463
:102CD0000E9488161092E9008091F000886080932D
:102CE000F000CD2BCF70C093E900FF91EF91DF9101
:102CF000CF91BF91AF919F918F917F916F915F9194
:102D00004F913F912F910F900FBE0F901F901895EC
:102D10001F93CF93DF93CDB7DEB7AA970FB6F89482
:102D2000DEBF0FBECDBFE7E5F3E088E08E0F9091E8
:102D3000F10091938E13FBCF0E942C128091E8003A
:102D400083FF1FC18091570390915803492F50E092
:102D50004A30510508F015C1FA01E156FF4F0C94B5
:102D6000662D803881F0823809F00BC180915B03B9
:102D70008F708093E9008091EB0085FB882780F9B4
:102D80001092E90006C08091530390915403911171
:102D900082609091E800977F9093E8008093F10023
:102DA0001092F100C8C0282F2D7F09F0EAC08823B7
:102DB00019F0823061F0E5C080915903813009F04B
:102DC000E0C0933009F080E0809354032BC08091E1
:102DD0005903811127C080915B038F7009F4D1C022
:102DE0008093E9002091EB0020FF1CC0933021F478
:102DF0008091EB00806214C09091EB009061909301
:102E0000EB0021E030E0A90102C0440F551F8A9574
:102E1000E2F74093EA001092EA008091EB008860AC
:102E20008093EB001092E9008091E800877F86C0D4
:102E30008111A7C0109159031F778091E30080781A
:102E4000812B8093E3008091E800877F8093E800E6
:102E50000E94A6148091E80080FFFCCF8091E300DF
:102E600080688093E300111102C082E001C083E01A
:102E70008093560386C08058823008F082C08091CB
:102E8000590390915A038C3D53E0950779F583E0FF
:102E90008A838AE289834FB7F894DE01139620E093
:102EA0003EE051E2E32FF0E050935700E49120FF21
:102EB00003C0E295EF703F5FEF708E2F90E0EA3035
:102EC00010F0C79601C0C0968D939D932F5F24315B
:102ED00049F74FBF8091E800877F8093E8006AE25E
:102EE00070E0CE0101960E94AD1314C0AE014F5F99
:102EF0005F4F60915B030E94F412BC01892B09F4BF
:102F000040C09091E800977F9093E80089819A8172
:102F10000E9410148091E8008B778093E80031C004
:102F2000803879F58091E800877F8093E800809170
:102F300052038093F1008091E8008E778093E8003F
:102F40000E94A6141EC081111CC09091590392309A
:102F5000C0F48091E800877F8093E800909352034B
:102F60000E94A61480915203811106C08091E30053
:102F700087FD02C081E001C084E0809356030E9477
:102F800018128091E80083FF0AC08091E800877FD3
:102F90008093E8008091EB0080628093EB00AA961A
:102FA0000FB6F894DEBF0FBECDBFDF91CF911F915A
:102FB00008959093EA028093E90208958091E902CE
:102FC0009091EA020895E091E902F091EA023097C7
:102FD00021F00190F081E02D099480E00895EF92B6
:102FE000FF920F931F93CF93DF93E091E902F0914B
:102FF000EA023097B1F18C010280F381E02D09954E
:103000008091410382FF2DC080FF04C088E596E0D7
:103010000E94E106E80118E082E5E82E86E0F82E3D
:103020008091410380FF0BC088811F928F93FF9294
:10303000EF920E947A070F900F900F900F9011500F
:1030400021961111EDCF8091410380FF0AC080E5E8
:1030500096E0DF91CF911F910F91FF90EF900C942C
:10306000E106DF91CF911F910F91FF90EF900895AE
:10307000E091E902F091EA02309721F00480F581B5
:10308000E02D09940895CF93DF93EC018091E7023E
:103090009091E802C817D90709F1D093E802C093CC
:1030A000E702E091E902F091EA023097B9F0068078
:1030B000F781E02DCE0109958091410382FF0EC07A
:1030C00080FF0CC0DF93CF9382E496E09F938F93B1
:1030D0000E947A070F900F900F900F90DF91CF9181
:1030E0000895CF93DF93EC018091E5029091E60281
:1030F000C817D90709F1D093E602C093E502E09121
:10310000E902F091EA023097B9F00084F185E02DF0
:10311000CE0109958091410382FF0EC080FF0CC053
:10312000DF93CF9382E396E09F938F930E947A0779
:103130000F900F900F900F90DF91CF9108950E9404
:103140006E240C949607CF92DF92EF92FF920F932A
:103150001F93CF93DF9300D000D000D0CDB7DEB760
:103160000E94C1078CEEC82E82E0D82E00E010E04D
:10317000E02E802F0E949208F60141916F01F42EFB
:10318000F826B1F40F5F1F4F0830110589F78FEF54
:1031900089838A831B820E9477248160782F9D8394
:1031A0008C8349815A816B818D810E94971947C018
:1031B0009091410391FF04C08E830E9463198E8118
:1031C00020E030E04F2D50E0922FBA01022E02C0D5
:1031D000759567950A94E2F760FF2BC02983EA8210
:1031E00021E030E0690102C0CC0CDD1C9A95E2F7C9
:1031F00090E08C219D21892B09F420E02B830E94F3
:1032000077248160782F9D838C8349815A816B81DB
:103210008D810E94971949815A816B817C818D81B2
:103220000E94F123F801E451FD4F8081C826C0823D
:1032300006C02F5F3F4F2830310531F6A3CF0E94E3
:10324000F0230E9464271091EB020E94E3171817E5
:1032500041F10E94E3178093EB029091410392FFAA
:103260000EC090FF0CC01F928F9383E696E09F9351
:103270008F930E947A070F900F900F900F9080917C
:10328000EB0226960FB6F894DEBF0FBECDBFDF91DE
:10329000CF911F910F91FF90EF90DF90CF900C9402
:1032A000022426960FB6F894DEBF0FBECDBFDF9185
:1032B000CF911F910F91FF90EF90DF90CF900895E5
:1032C0000C949F080895EF92FF920F931F93CF9352
:1032D000DF938CE796E00E94E106C0E0D0E08EE24A
:1032E000E82E81E0F82E0EE616E08C2F0E94920860
:1032F0000E94DA23FF92EF921F928F93DF93CF9376
:103300001F930F930E947A0721968DB79EB7089658
:103310000FB6F8949EBF0FBE8DBFC830D10529F7F8
:10332000DF91CF911F910F91FF90EF900895CF9370
:10333000DF93CDB7DEB72B970FB6F894DEBF0FBE85
:10334000CDBF942F4F83252F588769877A878B8726
:103350004A855B85452B21F02F3F09F59F3FF9F406
:10336000DE01119686E0FD0111928A95E9F785E06C
:10337000FE01379601900D928A95E1F749815A81B5
:103380006B817C818D819E810E9472202B960FB66D
:10339000F894DEBF0FBECDBFDF91CF9108954F816E
:1033A000588569857A858B850E94F123D9CFCF9383
:1033B000882309F465C0C82F8CEF8C0F813A20F068
:1033C00080E58C0F8E3248F48C2F0E948A2A81115E
:1033D00057C08C2F0E94FD220CC080E28C0F8830D9
:1033E00058F4C77081E001C0880FCA95EAF70E94BF
:1033F0003C23CF910C9480238BE58C0F833078F4A1
:10340000C53A29F0C63A31F083E890E005C081E87A
:1034100090E002C082E890E0CF910C94431888E5D8
:103420008C0F853168F5C83A89F0C93A91F0CA3AEB
:1034300099F0CB3AA1F0CC3AA9F0CD3AB1F0CE3A1E
:10344000B9F0CF3AC1F080E090E017C082EE90E092
:1034500014C089EE90E011C08AEE90E00EC085EBBA
:1034600090E00BC086EB90E008C083EB90E005C0D5
:1034700084EB90E002C087EB90E0CF910C94711840
:10348000CF910895882349F19CEF980F913A20F04D
:1034900090E5980F9E3218F40E941A230DC090E216
:1034A000980F983058F4877091E001C0990F8A9571
:1034B000EAF7892F0E9442230C9480239BE5980F02
:1034C000933020F480E090E00C944318885A8531C2
:1034D00020F480E090E00C9471180895882321F086
:1034E0000E943C230C9480230895882321F00E949D
:1034F00042230C9480230895BF92CF92DF92EF92E3
:10350000FF920F931F93CF93DF9300D000D000D092
:10351000CDB7DEB725E0FC01DE01119601900D92DA
:103520002A95E1F7FC0140813181F28025812295C5
:103530002F7063817481672B09F4FEC23F3F19F439
:103540004F3F09F4F9C26C0149833A8389819A811A
:103550002E830E94BC22182FB92E0E94BB220E94EB
:10356000CB21EB2DE295EF70F0E0E755FF4F2E8178
:103570000C94662D8B2D807F9B2D9F70092F8823A7
:1035800011F00295007FFF2049F0002309F481C269
:10359000802F0E944F230E9480237BC2812F0E9494
:1035A000421A002309F4C8C2802F0E945523269690
:1035B0000FB6F894DEBF0FBECDBFDF91CF911F9144
:1035C0000F91FF90EF90DF90CF90BF900C948023ED
:1035D0008B2D807F9B2D9F70092F803211F00295DB
:1035E000007F112319F0113009F12AC0FF20B1F03A
:1035F000802F222351F1213041F526960FB6F89401
:10360000DEBF0FBECDBFDF91CF911F910F91FF9015
:10361000EF90DF90CF90BF900C945F23222319F09E
:10362000213009F489C20E9468232DC0FF20F1F0E7
:10363000263008F081C20E943923802329F023C05C
:10364000FF20F9F0211116C0802F26960FB6F894AE
:10365000DEBF0FBECDBFDF91CF911F910F91FF90C5
:10366000EF90DF90CF90BF900C946E1A253008F049
:1036700063C209C0F601858180FF0BC28F7085830C
:10368000E3CF21111BC2802F82C12B2D26952695B9
:10369000237030E02115310521F021303105D1F0C2
:1036A0004BC2FF2021F0812F9B2D937002C080E040
:1036B00090E026960FB6F894DEBF0FBECDBFDF9127
:1036C000CF911F910F91FF90EF90DF90CF90BF901F
:1036D0000C944318FF2021F0812F9B2D937002C082
:1036E00080E090E026960FB6F894DEBF0FBECDBF07
:1036F000DF91CF911F910F91FF90EF90DF90CF90CE
:10370000BF900C947118812FFF2019F00E94EA25B8
:1037100002C00E94522626960FB6F894DEBF0FBE56
:10372000CDBFDF91CF911F910F91FF90EF90DF9070
:10373000CF90BF900C94D7268B2D837009F07BC05F
:10374000F110FAC1812F829586958770880F880FB6
:10375000912F9F70C92ED12CE12CF12C082E04C082
:10376000CC0CDD1CEE1CFF1C0A94D2F714FF12C017
:103770004FE050E060E070E004C0440F551F661F4A
:10378000771F8A95D2F7CB01BA0160957095809525
:10379000909503C060E070E0CB012B2D2695269517
:1037A0002370422F50E042305105D9F0433051058B
:1037B00069F16C297D298E299F294130510551F1EC
:1037C00026960FB6F894DEBF0FBECDBFDF91CF9126
:1037D0001F910F91FF90EF90DF90CF90BF900C94CE
:1037E000E0216C297D298E299F2926960FB6F89411
:1037F000DEBF0FBECDBFDF91CF911F910F91FF9024
:10380000EF90DF90CF90BF900C94F2210E94E021C6
:10381000C701B60126960FB6F894DEBF0FBECDBF26
:10382000DF91CF911F910F91FF90EF90DF90CF909C
:10383000BF900C94CE21FF2019F08B2D817001C018
:103840008695882309F478C1812F829586958770A3
:10385000880F880F912F9F70C92ED12CE12CF12C4D
:10386000082E04C0CC0CDD1CEE1CFF1C0A94D2F701
:1038700014FF12C04FE050E060E070E004C0440F5D
:10388000551F661F771F8A95D2F7CB01BA01609545
:1038900070958095909503C060E070E0CB012B2D72
:1038A000269526952370422F50E042305105D9F0DD
:1038B0004330510569F16C297D298E299F294130BA
:1038C000510551F126960FB6F894DEBF0FBECDBF5D
:1038D000DF91CF911F910F91FF90EF90DF90CF90EC
:1038E000BF900C9497226C297D298E299F292696BA
:1038F0000FB6F894DEBF0FBECDBFDF91CF911F9101
:103900000F91FF90EF90DF90CF90BF900C94A92281
:103910000E949722C701B60126960FB6F894DEBF23
:103920000FBECDBFDF91CF911F910F91FF90EF9010
:10393000DF90CF90BF900C948522103FC9F128F4FE
:1039400080E4810F803250F09FC0123F09F461C0C3
:1039500008F44AC0133F09F471C096C0012F0071EA
:103960008B2D8F71FF2051F00E941E22812F00238A
:1039700019F08295807F69CE8F7067CE0E943F22BA
:10398000812F002319F08295807F01C08F702696C9
:103990000FB6F894DEBF0FBECDBFDF91CF911F9160
:1039A0000F91FF90EF90DF90CF90BF900C94751A1D
:1039B000FF20B1F0253008F0BFC08B2D8F71269607
:1039C0000FB6F894DEBF0FBECDBFDF91CF911F9130
:1039D0000F91FF90EF90DF90CF90BF900C946422F6
:1039E000263008F0A9C0E9CFFF20A9F08B2D8F71F8
:1039F00026960FB6F894DEBF0FBECDBFDF91CF91F4
:103A00001F910F91FF90EF90DF90CF90BF900C949B
:103A10001E22FF2059F38B2D8F7126960FB6F89436
:103A2000DEBF0FBECDBFDF91CF911F910F91FF90F1
:103A3000EF90DF90CF90BF900C943F22FF2099F041
:103A40008B2D8F7126960FB6F894DEBF0FBECDBFBB
:103A5000DF91CF911F910F91FF90EF90DF90CF906A
:103A6000BF900C94092226960FB6F894DEBF0FBEC5
:103A7000CDBFDF91CF911F910F91FF90EF90DF901D
:103A8000CF90BF900C940422FF20A9F0222309F4C8
:103A9000ADCF812F26960FB6F894DEBF0FBECDBFF7
:103AA000DF91CF911F910F91FF90EF90DF90CF901A
:103AB000BF900C94D719222309F4ADCF812F2696FD
:103AC0000FB6F894DEBF0FBECDBFDF91CF911F912F
:103AD0000F91FF90EF90DF90CF90BF900C94421A1F
:103AE0004B2D4F70612FC6010E94642526960FB69C
:103AF000F894DEBF0FBECDBFDF91CF911F910F9124
:103B0000FF90EF90DF90CF90BF900C9416214B2D3B
:103B10004F70612FC60126960FB6F894DEBF0FBE18
:103B2000CDBFDF91CF911F910F91FF90EF90DF906C
:103B3000CF90BF900C94672526960FB6F894DEBF01
:103B40000FBECDBFDF91CF911F910F91FF90EF90EE
:103B5000DF90CF90BF9008950E945C230E942B239A
:103B60000E9480230E9409280E94D72680E090E0CE
:103B70000E94431880E090E00C9471180E944C233E
:103B80000C94AC1D0E94BC22292F22952F7030E08E
:103B90002C3031054CF42A303105C4F4225031095F
:103BA0002230310540F023C02C303105D1F02F30C8
:103BB0003105B9F01CC0853A28F48430B0F4823065
:103BC00028F413C090E2980F983078F0883E30F4D3
:103BD000803E58F48450813A50F407C0803F39F455
:103BE00004C093FB882780F9089581E0089580E060
:103BF0000895CF93DF9300D000D01F92CDB7DEB7EA
:103C00000F900F900F900F900F90DF91CF9108952C
:103C1000CF93DF9300D000D000D0CDB7DEB726968B
:103C20000FB6F894DEBF0FBECDBFDF91CF910895E0
:103C30001F93CF93DF93C091F40216E08091F502B9
:103C4000C81799F0D0E01C9FF0011D9FF00D1124C2
:103C5000EA50FD4F40815181628173818481958159
:103C60000E94081E2196C770E9CFDF91CF911F9166
:103C70000895409126035091270360912803709185
:103C8000290380912A0390912B030C94081E8091A4
:103C90002B0382958F7009F054C0809128038823EC
:103CA00009F44FC08091F402A091F50260912603BF
:103CB000709127034091290350912A03B6E08A1797
:103CC00009F43FC090E041155105C1F17F3F11F467
:103CD0006F3FA1F1B89FF001B99FF00D1124EA5098
:103CE000FD4F218172132AC02081621327C02281D7
:103CF000211124C0238134812417350710F4215069
:103D00003109241B350B2C323140C0F420912B0398
:103D10002F70206120932B0326E0289FF001299F1C
:103D2000F00D1124E550FD4F80818F7080618083FC
:103D300086E293E00E947C1A0C94181E019687700C
:103D4000BECF0895CF92DF92EF92FF920F931F9311
:103D5000CF93DF93CDB7DEB762970FB6F894DEBF8F
:103D60000FBECDBF8C0185E0F801DE011D960190EC
:103D70000D928A95E1F7D8014C9111965C911197BB
:103D800012966C9112971396CD90DC901497309107
:103D90002603709127038091290390912A030097AD
:103DA00009F473C17F3F19F43F3F09F46EC1E090FD
:103DB0002803EE2009F4C5C020912B03C816D906AC
:103DC00050F0F601E81BF90BCF01FF24F3948C327D
:103DD0009140C8F009C0809590958C0D9D1DFF24E1
:103DE000F3948C32914078F0F12C207F09F0C6C01A
:103DF0007C2DD98AC88A89890E94F91D86E293E0C0
:103E00000E947C1AB1C0822F807F09F045C07513D3
:103E100013C0341311C061110FC02F7020612093A3
:103E20002B030E94391E86E293E00E947C1A809147
:103E30002B03F80185832EC0CD2819F15F3F11F4C3
:103E40004F3FF9F0F62E61111CC08091F4022091D1
:103E5000F50236E0821709F45BC090E0389FF0016C
:103E6000399FF00D1124EA50FD4F7181571306C0A0
:103E70007081471303C07281711103C0019687706E
:103E8000E9CFF62E662309F41DC180912B038160D2
:103E900080932B03F12C16C1751309C0341307C08E
:103EA000611105C080912B03F8018583C8C04D873F
:103EB0005E878D859E856A8B0E94C21D6A898823D4
:103EC000E1F16623D1F120912B03822F82958F702F
:103ED00090E0029774F080912603909127039887D1
:103EE0008F831986DB86CA862C87CE0107960E94AF
:103EF0007C1A86E0F801A6E2B3E001900D928A9563
:103F0000E1F70E94471E0E94391EFF24F394DAC095
:103F10004D875E878D859E850E94BC22292F229524
:103F20002F7030E0223031050CF0BFC09F7009F0D7
:103F3000B9C0805E883008F4C5C0C8010E947C1AF0
:103F4000E4CFC816D90608F453C0F601E81BF90BF4
:103F5000CF018C32914008F453C0F12C7C2DD98ACA
:103F6000C88A89890E94F91DE6E2F3E086E0DF0154
:103F70001D928A95E9F70E94391EA4C0751314C0DA
:103F8000341312C0611110C080912B03F801858396
:103F9000C8010E947C1A86E0E6E2F3E0DF011D9290
:103FA0008A95E9F7FE2C8EC04D875E878D859E85AC
:103FB0006A8B0E94C21D6A89882309F4BECF6623DA
:103FC00009F4BBCF20912B03822F82958F7090E054
:103FD00002970CF48ECF80912603909127039A8349
:103FE00089831B82DD82CC822E83CE0101967FCF16
:103FF000809590958C0D9D1D8C32914008F0ADCF31
:10400000F62E662309F499CF75132EC034132CC0F5
:1040100020912B0320FD1FC0822F82958F70D9F035
:10402000D80115962C9315978F3049F08F5F982FF4
:104030009295907F822F8F70892B15968C93C80153
:104040000E947C1A86E0F801A6E2B3E001900D928E
:104050008A95E1F790CF86E0F801A6E2B3E00190FF
:104060000D928A95E1F72EC04D875E878D859E85DE
:104070000E94C21D81113DCF80912B0381608093EE
:104080002B03C8010E947C1A1DC0662309F455CF7A
:104090004D875E878D859E850E94C21D882309F409
:1040A0004CCF27CF811145CF0DC0243031050CF006
:1040B00044CF9F7009F43DCFD80115969C91907F15
:1040C00009F037CF8F2D62960FB6F894DEBF0FBE82
:1040D000CDBFDF91CF911F910F91FF90EF90DF90B7
:1040E000CF9008951F93CF93DF93CDB7DEB72C9772
:1040F0000FB6F894DEBF0FBECDBF4F8358876987D8
:104100007A878B879C87CE0107960E94A21E882300
:1041100069F08F8198852A853B85232BF1F19F3F9C
:1041200009F063C08F3F09F060C037C086E0FE0130
:104130003796DE01119601900D928A95E1F76F8115
:104140007885EA85FB85309741F17F3F11F46F3F19
:1041500021F12091F50230E0C9010196877099277D
:104160004091F40250E08417950709F447C0698331
:104170007A83FD83EC8396E0929FD001939FB00DEC
:104180001124AA50BD4FFE01319601900D929A95CF
:10419000E1F78093F5020E94181E16E08091F40268
:1041A0009091F5028917C1F1189FC00111248A501E
:1041B0009D4F0E94A21E882379F1E091F4021E9F78
:1041C000F0011124EA50FD4F4081518162817381D9
:1041D000848195810E94081E8091F40290E00196EE
:1041E000877099278093F402D9CF4F8158856985CC
:1041F0007A858B859C850E94081ECFCF0E94BE1DAC
:104200001092F5021092F402E6E2F3E086E0DF019C
:104210001D928A95E9F7C1CF2C960FB6F894DEBFB0
:104220000FBECDBFDF91CF911F910895DF92EF9226
:10423000FF920F931F93CF93DF93FC01892B09F417
:104240008AC0E12CF12CDD24D394EF0121968491D6
:10425000853709F461C058F4843708F04EC08430C3
:1042600008F06AC08130D1F0823071F174C08837B3
:1042700009F45DC050F4863709F455C0873709F05A
:104280006AC08E2D0E94492354C09CE7980F903736
:1042900008F061C08F770E94421A50C08F010E5FF4
:1042A0001F4FFE01849190E2980F983050F4877070
:1042B000FD2D01C0FF0F8A95EAF78F2F0E944F2333
:1042C00014C00E94D71913C08F010E5F1F4FFE014B
:1042D000C49180E28C0F883060F4C7708D2D01C0CE
:1042E000880FCA95EAF70E9455230E948023E801AF
:1042F00025C08C2F0E94421AFACF9F012E5F3F4F9C
:10430000FE01C491CC2369F08FE99FE00197F1F79A
:1043100000C00000C150F6CF9F012E5F3F4FFE014D
:10432000F490E9010BC00E943923E82E07C00E94D7
:104330004C230E94802302C00E94D7198F2D88230E
:1043400041F0EFE9FFE03197F1F700C00000815044
:10435000F6CFFE017ACFDF91CF911F910F91FF90A1
:10436000EF90DF9008956093300370933103809352
:104370003203909333030E9400240C94AC1D60938D
:104380002C0370932D0380932E0390932F030E9490
:1043900001240C94AC1D08950C94B3210F931F932A
:1043A0000091300310913103209132033091330397
:1043B000602B712B822B932B1F910F910C94B321A7
:1043C0000F931F930091300310913103209132031A
:1043D0003091330360237123822393231F910F9124
:1043E0000C94B3210F931F9300913003109131036C
:1043F000209132033091330360277127822793275E
:104400001F910F910C94B32160E070E0CB010C94EC
:10441000BF210F931F9341E050E060E070E08A01FC
:104420009B0104C0000F111F221F331F8A95D2F772
:10443000C901B8011F910F910C94BF210F931F93D5
:1044400041E050E060E070E004C0440F551F661F7B
:10445000771F8A95D2F780912C0390912D03A0911C
:104460002E03B0912F038A019B01082B192B2A2BB5
:104470003B2BC901B8011F910F910C94BF210F93E1
:104480001F9341E050E060E070E004C0440F551F0E
:10449000661F771F8A95D2F7409550956095709565
:1044A00080912C0390912D03A0912E03B0912F03A6
:1044B0008A019B01082319232A233B23C901B80140
:1044C0001F910F910C94BF210F931F9341E050E077
:1044D00060E070E004C0440F551F661F771F8A9587
:1044E000D2F780912C0390912D03A0912E03B091CF
:1044F0002F038A019B01082719272A273B27C90177
:10450000B8011F910F910C94BF210F931F9300913D
:104510002C0310912D0320912E0330912F03602B3B
:10452000712B822B932B1F910F910C94BF210F9312
:104530001F9300912C0310912D0320912E03309195
:104540002F0360237123822393231F910F910C94D7
:10455000BF210F931F9300912C0310912D032091E5
:104560002E0330912F0360277127822793271F91F5
:104570000F910C94BF210895CF92DF92EF92FF929A
:104580000F931F93CF93DF938C01C0903003D09093
:104590003103E0903203F090330340912C035091AB
:1045A0002D0360912E0370912F03C42AD52AE62A89
:1045B000F72ACFE1D0E0D701C6010C2E04C0B69592
:1045C000A795979587950A94D2F780FF07C0B80101
:1045D0008C2F0E943A258130910531F4219758F7AC
:1045E000B80180E00E943A25DF91CF911F910F9191
:1045F000FF90EF90DF90CF900895209121013091AE
:104600002201F90132969FEF40E05191581789F04D
:104610009F3F19F4511101C0942F4F5F4630A9F705
:104620009F3F39F0F901E90FF11D97FDFA9582835B
:10463000089508952091210130912201F9013296C7
:10464000285F3F4F9081981301C010823196E21786
:10465000F307C1F7089581E090E0E0912101F09126
:104660002201E80FF91F1082019688309105A9F701
:10467000089580914003089590914003892B809381
:1046800040030895809590914003892380934003CF
:1046900008958093400308951092400308959091E7
:1046A0003F03892B80933F030895809590913F03AA
:1046B000892380933F03089510923F0308958093C8
:1046C00036030E9477249093350380933403089532
:1046D000109236031092350310923403089580919E
:1046E000210190912201FC0131969C01285F3F4FEE
:1046F00080E0919191118F5FE217F307D1F7089550
:10470000E0912101F0912201809140038083E091AA
:104710002101F0912201908180913F03892B8083B8
:10472000809136038823D9F10E94772420913403A5
:10473000309135038217930748F00E947724209127
:10474000340330913503821B930B0AC00E947724F7
:10475000209134033091350320953095820F931FBB
:104760008C32914070F08091410380FF08C08AE84C
:1047700096E09F938F930E947A070F900F900E946C
:104780006823E0912101F09122019081809136030C
:10479000892B80830E946F2381110E94682380915E
:1047A0002101909122010C94EF1790939B0180932B
:1047B0009A0108958295982F9C7C392F36953695CD
:1047C000282F237344E0249FC0011124932F982B9A
:1047D000292F2A7A2695892F8575880F822B08958F
:1047E0000895CF93DF9300D000D01F92CDB7DEB7EE
:1047F0000F900F900F900F900F90DF91CF91089531
:10480000089508950C94601980915603843021F125
:104810001092420320E488E190E00FB6F894A89546
:10482000809360000FBE2093600083B7817F846017
:1048300083BF83B7816083BF7894889583B78E7F69
:1048400083BF0FB6F894A89580916000886180932B
:104850006000109260000FBE0895CF930E949B08E5
:104860000E94C1070E949D08C0E08C2F0E94920800
:10487000811104C0CF5FC830C1F701C081E0CF9182
:1048800008950E9462190C94BE1D1F920F920FB6DC
:104890000F9211248F939F93AF93BF938091420304
:1048A000811113C08091430390914403A09145036B
:1048B000B09146034196A11DB11D8093430390938F
:1048C0004403A0934503B0934603BF91AF919F91DA
:1048D0008F910F900FBE0F901F90189582E084BDAE
:1048E00093E095BD9AEF97BD80936E0008952FB722
:1048F000F8948091430390914403A0914503B091B3
:1049000046032FBF08952FB7F89460914303709129
:10491000440380914503909146032FBF0895CF92A1
:10492000DF92EF92FF920F931F932FB7F89440916D
:1049300043035091440360914503709146032FBF98
:104940006A017B01EE24FF248C0120E030E0C016D8
:10495000D106E206F30610F4415051099A01281BD2
:10496000390BC9011F910F91FF90EF90DF90CF900D
:104970000895CF92DF92EF92FF920F931F932FB77C
:10498000F894C0904303D0904403E0904503F09026
:1049900046032FBF97018601061B170B280B390B07
:1049A000C616D706E806F90618F0C901B80106C010
:1049B000C901B80161507109810991091F910F91D5
:1049C000FF90EF90DF90CF9008951F920F920FB657
:1049D0000F9211248F939F93AF93BF9380914303C2
:1049E00090914403A0914503B09146030196A11D07
:1049F000B11D8093430390934403A0934503B09368
:104A00004603BF91AF919F918F910F900FBE0F9072
:104A10001F9018950E94F714F8942FEF87EA91E6FB
:104A2000215080409040E1F700C0000087E090EB0B
:104A3000DC0180935F0390936003A0936103B093C4
:104A400062039CE088E10FB6F894A895809360001B
:104A50000FBE90936000FFCF28E0929FF0011124D9
:104A6000E80FF11DEE58FE4F9491892F8F709295AB
:104A70009F700895CF93C82FCB010E942C25282F1B
:104A800030E080E1989FA0011124422B532B403845
:104A9000510519F480E090E015C09770E92FF0E01F
:104AA00088E0C89FE00DF11D112484E0EE0FFF1F88
:104AB0008A95E1F7E20FF31FEE0FFF1FE050F84970
:104AC00085919491CF91089580E090E008950895A4
:104AD0008091490380FF0BC06091260185E0689FAB
:104AE000B001112475956795759567952BC081FF69
:104AF00009C06091260185E0689FB0011124759579
:104B0000679520C082FF07C06091260185E0689FFD
:104B1000B001112417C090914A039923D1F06091FC
:104B20002501961788F72091260185E0289F90019E
:104B30001124929FA001939F500D112470E0CA018F
:104B40000E94302D6038710540F46115710539F00F
:104B500002C065E070E0862F08958FE7089581E038
:104B600008958091490380FF08C06091240170E09E
:104B7000759567957595679521C081FF06C0609111
:104B8000240170E07595679519C082FF04C060919B
:104B9000240170E010C090914A039923C1F0609104
:104BA00023019617A0F780912401899FC001112449
:104BB00070E00E94302D6038710528F46115710590
:104BC00021F0862F08958FE7089581E0089561E030
:104BD00070E0F4CF803F21F40E946825819504C0E5
:104BE000813F29F40E94682580934D030895823FF8
:104BF00021F40E946825819504C0833F29F40E9416
:104C0000682580934C030895893F19F40E94B125CB
:104C100005C08A3F31F40E94B125819580934E03EF
:104C200008958B3F21F40E94B125819504C08C3FEB
:104C300029F40E94B12580934F030895843F21F405
:104C400080914B03816017C0853F21F480914B0315
:104C5000826011C0863F21F480914B0384600BC0B9
:104C6000873F21F480914B03886005C0883F31F471
:104C700080914B03806180934B0308958D3F21F415
:104C80008091490381600BC08E3F21F480914903DC
:104C9000826005C08F3F29F480914903846080932E
:104CA00049030895803F39F480914D0387FF6CC01C
:104CB00010924D0369C0813F29F480914D0318166D
:104CC000BCF362C090914C03823F29F497FF5CC013
:104CD00010924C0359C0833F19F41916CCF354C0F9
:104CE000893F41F480914E0318160CF04DC010928C
:104CF0004E034AC08A3F29F480914E0387FF44C087
:104D0000F6CF8B3F39F480914F0387FF3DC010925F
:104D10004F033AC08C3F29F480914F031816BCF31F
:104D200033C0843F21F480914B038E7F17C0853FB1
:104D300021F480914B038D7F11C0863F21F4809137
:104D40004B038B7F0BC0873F21F480914B03877F00
:104D500005C0883F31F480914B038F7E80934B03D5
:104D600013C08D3F21F4809149038E7F0BC08E3F8D
:104D700021F4809149038D7F05C08F3F29F48091F4
:104D800049038B7F8093490380914C0381110EC0AE
:104D900080914D0381110AC080914E03811106C09C
:104DA00080914F03811102C010924A0308958091AF
:104DB000410383FF7EC083EC96E00E94E106809170
:104DC0004B031F928F938EEB96E09F938F930E94DD
:104DD0007A078CEB96E00E94E10680914C03282F25
:104DE000082E000C330B3F938F9389EB96E09F9333
:104DF0008F930E947A0787EB96E00E94E1068091EC
:104E00004D03282F082E000C330B3F938F9384EB18
:104E100096E09F938F930E947A0782EB96E00E9420
:104E2000E10680914E03282F082E000C330B3F9390
:104E30008F938FEA96E09F938F930E947A078DEA73
:104E400096E00E94E10680914F03282F082E000C67
:104E5000330B3F938F938AEA96E09F938F930E9440
:104E60007A0787EA96E00E94E10680914A031F9242
:104E70008F9384EA96E09F938F930E947A0782EA49
:104E800096E00E94E106809149031F928F938FE97B
:104E900096E09F938F930E947A078CE996E00E9498
:104EA000E1068DB79EB74C960FB6F8949EBF0FBE25
:104EB0008DBF8BE493E00E9438180E947724909372
:104EC00048038093470308951F93CF93DF93809106
:104ED0004703909148030E948F24AC0190914A03AC
:104EE000992321F02091270130E006C0209128016C
:104EF0008AE0289F900111244217530708F485C0C7
:104F000080914C03C0914D03D0914E0310914F03FB
:104F1000811107C0C11175C0D11173C0111171C0C9
:104F200074C09F3F19F09F5F90934A03181624F4B2
:104F30000E94682580934C0380914C0387FF05C035
:104F40000E946825819580934C031C1624F40E94CE
:104F5000682580934D0380914D0387FF05C00E9413
:104F60006825819580934D0360914C03662331F150
:104F7000C0914D03CC2311F1062E000C770B880B4A
:104F8000990B0E94172C23E333E343E35FE30E9472
:104F90007B2C0E94DF2B60934C036C2FCC0F770B84
:104FA000880B990B0E94172C23E333E343E35FE361
:104FB0000E947B2C0E94DF2B60934D031D1624F46E
:104FC0000E94B12580934E0380914E0387FF05C058
:104FD0000E94B125819580934E03111624F40E94FE
:104FE000B12580934F0380914F0387FF05C00E9436
:104FF000B125819580934F03DF91CF911F910C9440
:10500000D7269F3F09F08FCF97CFDF91CF911F9188
:105010000895EBE4F3E085E0DF011D928A95E9F75E
:1050200010924A0310924903089586EE98E00E9478
:10503000E1061F9281E08F931F9285E08F9388E9AC
:1050400098E09F938F930E947A070F900F900F9094
:105050000F900F900F9008958330E9F128F481307C
:1050600061F0823009F10895853009F462C008F4D6
:1050700049C0863009F474C0089580912801262F14
:1050800030E0280F311D2F3F310524F4680F609365
:10509000280103C08FEF80932801809128011F927F
:1050A0008F9381ED97E072C080912701262F30E029
:1050B000280F311D2F3F310524F4680F609327011D
:1050C00003C08FEF80932701809127011F928F9358
:1050D0008FEB97E05BC080912601262F30E0280FF0
:1050E000311D2F3F310524F4680F6093260103C062
:1050F0008FEF80932601809126011F928F938CEA77
:1051000097E044C080912501262F30E0280F311D03
:105110002F3F310524F4680F6093250103C08FEF02
:1051200080932501809125011F928F9387E997E055
:105130002DC080912401262F30E0280F311D2F3FF4
:10514000310524F4680F6093240103C08FEF80932E
:105150002401809124011F928F938EE797E016C05F
:1051600080912301262F30E0280F311D2F3F31057C
:1051700024F4680F6093230103C08FEF8093230111
:10518000809123011F928F9383E697E09F938F93E3
:105190000E947A070F900F900F900F900895833020
:1051A00081F128F4813059F08230D1F008958530B2
:1051B00009F449C0B8F1863009F456C008958091C9
:1051C0002801681720F4861B8093280102C01092E2
:1051D0002801809128011F928F9384E597E054C0A5
:1051E00080912701681720F4861B8093270102C055
:1051F00010922701809127011F928F9382E497E0FC
:1052000043C080912601681720F4861B80932601F5
:1052100002C010922601809126011F928F938FE287
:1052200097E032C080912501681720F4861B809397
:10523000250102C010922501809125011F928F93B4
:105240008AE197E021C080912401681720F4861B31
:105250008093240102C010922401809124011F92A6
:105260008F9381E097E010C080912301681720F4AC
:10527000861B8093230102C0109223018091230199
:105280001F928F9386EE96E09F938F930E947A07EA
:105290000F900F900F900F900895CF93C82F1F92EB
:1052A0008F938BEE99E09F938F930E947A0781E012
:1052B00090E0A0E0B0E0BC01CD0104C0660F771F14
:1052C000881F991FCA95D2F70E94CC210F900F908A
:1052D0000F900F90CF910C94BE1DCF93873288F51D
:1052E0008E3108F00BC18E3009F487C0D8F48730B6
:1052F00009F460C08B3009F44FC0863009F002C158
:1053000080914103817F8E7F8093410380EF99E0FC
:105310000E94E10685EA9CE00E94E10681E080931C
:10532000510346C0863109F4B0C020F4803109F43D
:105330007AC0E8C0893109F491C08B3109F449C0C1
:10534000E1C0883349F150F4893209F4D5C085337E
:1053500009F4D2C0873209F0D5C0CEC0833409F435
:10536000CBC028F48A3308F4CDC08953C8C0883430
:1053700009F0C8C00E94BE1D84E99CE00E94E106BD
:105380002FEF83ED90E3215080409040E1F700C083
:1053900000000E940A250CC087E19AE041C08BE71B
:1053A0009CE00E94E106809141038160809341036B
:1053B000C1E0ADC080914103C82FC17080FFEFCF25
:1053C00087E89CE00E94E10680914103817F8E7F07
:1053D0003FC09091410391FBCC27C0F981E0C827E1
:1053E000892FC0FB81F980934103CC2319F08EE60D
:1053F0009CE029C080E69CE013C09091410392FBA1
:10540000CC27C0F981E0C827892FC0FB82F980939F
:105410004103CC2319F081E59CE015C081E49CE0B8
:105420000E94E106C5CF9091410393FBCC27C0F9C0
:1054300081E0C827892FC0FB83F980934103CC23E7
:1054400051F085E39CE00E94E10680914103816078
:10545000809341035CC088E29CE0E2CF89E19CE05C
:105460000E94E1068CEE9BE00E94E10685EB9BE04A
:105470000E94E10688E89BE00E94E10683E49BE04D
:105480000E94E10685E19BE0CBCF87E09BE00E9494
:10549000E1060E94E3171F928F938DEE9AE09F938F
:1054A0008F930E947A07809120011F928F9386ED3F
:1054B0009AE09F938F930E947A078091E4021F9253
:1054C0008F9383EC9AE09F938F930E947A070E94B8
:1054D00083249F938F937F936F938CEA9AE09F939B
:1054E0008F930E947A078DB79EB742960FB6F894B5
:1054F0009EBF0FBE8DBF5CCF80E001C08D510E946A
:105500004D2956CF8AEA9AE00E94E106C0E08C2F2E
:10551000CF910895CF93C82F80915103813071F0BE
:1055200020F0823009F44BC042C1E0912101F0919A
:1055300022018081823209F03CC107C0E091210143
:10554000F09122018081823261F48C2F0E94D20B73
:10555000811104C08C2F0E946D292FC081E090E042
:105560002CC08C2F0E94FF0D811126C0C431E1F0A8
:1055700070F4CB3081F0C031D1F40E94152883EE55
:1055800099E00E94E10682E08093510315C0C93280
:1055900059F0C83361F480EF99E00E94E10687EE8C
:1055A00099E00E94E10608C01092510304C181EE07
:1055B00099E00E94E106FFC081E08170FEC0C43224
:1055C00028F5CE3108F0C1C0CB30A1F1D0F4C730FE
:1055D00009F0D3C08EE18093280182E380932701F4
:1055E0008AE08093260184E18093250188E08093FE
:1055F000240188E28093230187E898E00E94E10675
:10560000BFC0C33149F1C431C1F0B7C0CB3409F4D4
:10561000A9C028F4C93289F0C83361F0AEC0C135E1
:1056200009F49EC0C23509F499C0CE3409F0A5C072
:105630006AE09EC00E941528A3C080915003882371
:1056400019F0109250039CC084E998E00E94E10692
:1056500081E080935103B1C08EE698E00E94E1069C
:105660008CE598E00E94E106809128011F928F93BB
:1056700089E598E09F938F930E947A0787E598E0E9
:105680000E94E10685E498E00E94E10680912701EE
:105690001F928F9382E498E09F938F930E947A07E2
:1056A00080E498E00E94E10681E398E00E94E10630
:1056B000809126011F928F938EE298E09F938F93A3
:1056C0000E947A078CE298E00E94E1068BE198E064
:1056D0000E94E106809125011F928F9388E198E056
:1056E0009F938F930E947A0786E198E00E94E106DB
:1056F00081E098E00E94E106809124011F928F933F
:105700008EEF97E09F938F930E947A078CEF97E03C
:105710000E94E10685EE97E00E94E1068091230158
:105720001F928F9382EE97E09F938F930E947A0748
:1057300080EE97E00E94E1068DB79EB748960FB6BF
:10574000F8949EBF0FBE8DBF1BC0CE51EC2FF0E072
:10575000E057FE4F80818093500312C061E003C088
:1057600061E006C06AE0809150030E942C2808C0C6
:10577000809150030E94CF2803C085E898E013C0B1
:1057800080915003882369F01F928F938FE798E0F0
:105790009F938F930E947A070F900F900F900F9016
:1057A00004C08CE798E00E94E10681E006C01092F8
:1057B000510380E002C080E000CFCF9108950E94A5
:1057C000E62B6894B1110C94752C08950E945A2C04
:1057D00088F09F5798F0B92F9927B751B0F0E1F0B2
:1057E000660F771F881F991F1AF0BA95C9F714C062
:1057F000B13091F00E94742CB1E008950C94742C97
:10580000672F782F8827B85F39F0B93FCCF386959A
:1058100077956795B395D9F73EF4909580957095F7
:1058200061957F4F8F4F9F4F0895E89409C097FB74
:105830003EF490958095709561957F4F8F4F9F4F67
:105840009923A9F0F92F96E9BB279395F6958795AB
:1058500077956795B795F111F8CFFAF4BB0F11F46E
:1058600060FF1BC06F5F7F4F8F4F9F4F16C0882315
:1058700011F096E911C0772321F09EE8872F762F4B
:1058800005C0662371F096E8862F70E060E02AF08C
:105890009A95660F771F881FDAF7880F9695879578
:1058A00097F9089557FD9058440F551F59F05F3FE1
:1058B00071F04795880F97FB991F61F09F3F79F032
:1058C00087950895121613061406551FF2CF4695B4
:1058D000F1DF08C0161617061806991FF1CF869536
:1058E0007105610508940895E894BB27662777271A
:1058F000CB0197F908950E948E2C0C94FF2C0E94E6
:10590000F12C38F00E94F82C20F0952311F00C9423
:10591000E82C0C94EE2C11240C94752C0E94522C23
:1059200070F3959FC1F3950F50E0551F629FF001F2
:10593000729FBB27F00DB11D639FAA27F00DB11D0B
:10594000AA1F649F6627B00DA11D661F829F222794
:10595000B00DA11D621F739FB00DA11D621F839F1B
:10596000A00D611D221F749F3327A00D611D231FF1
:10597000849F600D211D822F762F6A2F11249F573F
:1059800050409AF0F1F088234AF0EE0FFF1FBB1F42
:10599000661F771F881F91505040A9F79E3F510501
:1059A00080F00C94E82C0C94752C5F3FE4F3983E47
:1059B000D4F3869577956795B795F795E7959F5FAB
:1059C000C1F7FE2B880F911D9695879597F908953D
:1059D00097F99F6780E870E060E008959FEF80ECA2
:1059E000089500240A941616170618060906089545
:1059F00000240A9412161306140605060895092EAB
:105A00000394000C11F4882352F0BB0F40F4BF2B19
:105A100011F460FF04C06F5F7F4F8F4F9F4F089559
:105A2000991B79E004C0991F961708F0961B881FF0
:105A30007A95C9F780950895AA1BBB1B51E107C051
:105A4000AA1FBB1FA617B70710F0A61BB70B881F0E
:105A5000991F5A95A9F780959095BC01CD0108959D
:105A600097FB072E16F4009407D077FD09D00E940B
:105A70001C2D07FC05D03EF4909581959F4F08950D
:105A8000709561957F4F0895A1E21A2EAA1BBB1B4A
:105A9000FD010DC0AA1FBB1FEE1FFF1FA217B307FA
:105AA000E407F50720F0A21BB30BE40BF50B661F10
:105AB000771F881F991F1A9469F7609570958095D4
:105AC00090959B01AC01BD01CF010895EE0FFF1F22
:0C5AD0000590F491E02D0994F894FFCFAC
:105ADC0027092A092B092C092D092309A7098D0946
:105AEC0026092E090A019C108D116A11361102111A
:105AFC000137032808140A321E524E2D3432004C42
:105B0C00554641004F4646004F4E00434F4E4E0007
:105B1C00506F776572656400556E6174746163686B
:105B2C0065640044656661756C74004164647265FB
:105B3C007373656400436F6E6669677572656400A4
:105B4C003F0053757370656E64656400404D36227A
:105B5C00F205A5056F054D05D904F2040B052405C6
:0A5B6C000102030405060708090002
:106800000000000000000000040005000600070072
:10681000080009000A000B000C000D000E000F001C
:1068200010001100120013001400150016001700CC
:10683000180019001A001B001C001D001E001F007C
:10684000200021002200230024002500260027002C
:106850002800000035002B002C002D002E002F00FA
:1068600030002A00000033003400290036003700D1
:106870003800E00000000000000000000000000000
:106880000000000000000000000000000000000008
:1068900000000000000000000000000000000000F8
:1068A00000000000000000000000000000000000E8
:1068B00000000000000000000000000000000000D8
:1068C00000000000000000000000000000000000C8
:1068D00000000000000000000000000000000000B8
:1068E0000000000000000000310000000000000077
:1068F0000000E100E200E300F1A1E500E600E700AE
:106900000000000000000000EA4401000100E24431
:106910000100010001005500460054004A004B00F0
:10692000560057004700480001000100E9440100FB
:106930000100010001000100010001003A003B00DC
:106940003C003D003E003F0040004100420043004B
:10695000580000004C00390001004400450052007E
:1069600001000100000050004F0081404D004E002A
:1069700051000100000000000000000000000000C5
:106980000000000000000000000000000000000007
:1069900000000000000000000000000000000000F7
:1069A00000000000000000000000000000000000E7
:1069B00000000000000000000000000000000000D7
:1069C00000000000000000000000000000000000C7
:1069D00000000000000000000000000000000000B7
:1069E000000000000000000049000000000000005E
:1069F0000000010001000100010001000100010090
:00000001FF
